Archive member included to satisfy reference by file (symbol)

d:/ahl-gec-ide(4.26)º¬python/gcc/bin/../lib/gcc/arm-none-eabi/7.2.1/../../../../arm-none-eabi/lib/thumb/v7e-m/fpv4-sp/hard\libc_nano.a(lib_a-exit.o)
                              d:/ahl-gec-ide(4.26)º¬python/gcc/bin/../lib/gcc/arm-none-eabi/7.2.1/../../../../arm-none-eabi/lib/thumb/v7e-m/fpv4-sp/hard/crt0.o (exit)
d:/ahl-gec-ide(4.26)º¬python/gcc/bin/../lib/gcc/arm-none-eabi/7.2.1/../../../../arm-none-eabi/lib/thumb/v7e-m/fpv4-sp/hard\libc_nano.a(lib_a-impure.o)
                              d:/ahl-gec-ide(4.26)º¬python/gcc/bin/../lib/gcc/arm-none-eabi/7.2.1/../../../../arm-none-eabi/lib/thumb/v7e-m/fpv4-sp/hard\libc_nano.a(lib_a-exit.o) (_global_impure_ptr)
d:/ahl-gec-ide(4.26)º¬python/gcc/bin/../lib/gcc/arm-none-eabi/7.2.1/../../../../arm-none-eabi/lib/thumb/v7e-m/fpv4-sp/hard\libc_nano.a(lib_a-init.o)
                              d:/ahl-gec-ide(4.26)º¬python/gcc/bin/../lib/gcc/arm-none-eabi/7.2.1/../../../../arm-none-eabi/lib/thumb/v7e-m/fpv4-sp/hard/crt0.o (__libc_init_array)
d:/ahl-gec-ide(4.26)º¬python/gcc/bin/../lib/gcc/arm-none-eabi/7.2.1/../../../../arm-none-eabi/lib/thumb/v7e-m/fpv4-sp/hard\libc_nano.a(lib_a-memcpy-stub.o)
                              ./obj/flash.o (memcpy)
d:/ahl-gec-ide(4.26)º¬python/gcc/bin/../lib/gcc/arm-none-eabi/7.2.1/../../../../arm-none-eabi/lib/thumb/v7e-m/fpv4-sp/hard\libc_nano.a(lib_a-memset.o)
                              d:/ahl-gec-ide(4.26)º¬python/gcc/bin/../lib/gcc/arm-none-eabi/7.2.1/../../../../arm-none-eabi/lib/thumb/v7e-m/fpv4-sp/hard/crt0.o (memset)
d:/ahl-gec-ide(4.26)º¬python/gcc/bin/../lib/gcc/arm-none-eabi/7.2.1/../../../../arm-none-eabi/lib/thumb/v7e-m/fpv4-sp/hard\libc_nano.a(lib_a-strcmp.o)
                              ./obj/emuart.o (strcmp)
d:/ahl-gec-ide(4.26)º¬python/gcc/bin/../lib/gcc/arm-none-eabi/7.2.1/../../../../arm-none-eabi/lib/thumb/v7e-m/fpv4-sp/hard\libc_nano.a(lib_a-strlen.o)
                              ./obj/printf.o (strlen)
d:/ahl-gec-ide(4.26)º¬python/gcc/bin/../lib/gcc/arm-none-eabi/7.2.1/../../../../arm-none-eabi/lib/thumb/v7e-m/fpv4-sp/hard\libc_nano.a(lib_a-strncmp.o)
                              ./obj/emuart.o (strncmp)
d:/ahl-gec-ide(4.26)º¬python/gcc/bin/../lib/gcc/arm-none-eabi/7.2.1/thumb/v7e-m/fpv4-sp/hard\libgcc.a(_arm_addsubdf3.o)
                              ./obj/uart.o (__aeabi_dsub)
d:/ahl-gec-ide(4.26)º¬python/gcc/bin/../lib/gcc/arm-none-eabi/7.2.1/thumb/v7e-m/fpv4-sp/hard\libgcc.a(_arm_muldivdf3.o)
                              ./obj/uart.o (__aeabi_dmul)
d:/ahl-gec-ide(4.26)º¬python/gcc/bin/../lib/gcc/arm-none-eabi/7.2.1/thumb/v7e-m/fpv4-sp/hard\libgcc.a(_arm_cmpdf2.o)
                              ./obj/printf.o (__aeabi_dcmplt)
d:/ahl-gec-ide(4.26)º¬python/gcc/bin/../lib/gcc/arm-none-eabi/7.2.1/thumb/v7e-m/fpv4-sp/hard\libgcc.a(_arm_fixunsdfsi.o)
                              ./obj/uart.o (__aeabi_d2uiz)
d:/ahl-gec-ide(4.26)º¬python/gcc/bin/../lib/gcc/arm-none-eabi/7.2.1/thumb/v7e-m/fpv4-sp/hard\libgcc.a(_aeabi_uldivmod.o)
                              ./obj/printf.o (__aeabi_uldivmod)
d:/ahl-gec-ide(4.26)º¬python/gcc/bin/../lib/gcc/arm-none-eabi/7.2.1/thumb/v7e-m/fpv4-sp/hard\libgcc.a(_fixunsdfdi.o)
                              ./obj/printf.o (__aeabi_d2ulz)
d:/ahl-gec-ide(4.26)º¬python/gcc/bin/../lib/gcc/arm-none-eabi/7.2.1/thumb/v7e-m/fpv4-sp/hard\libgcc.a(_udivmoddi4.o)
                              d:/ahl-gec-ide(4.26)º¬python/gcc/bin/../lib/gcc/arm-none-eabi/7.2.1/thumb/v7e-m/fpv4-sp/hard\libgcc.a(_aeabi_uldivmod.o) (__udivmoddi4)
d:/ahl-gec-ide(4.26)º¬python/gcc/bin/../lib/gcc/arm-none-eabi/7.2.1/thumb/v7e-m/fpv4-sp/hard\libgcc.a(_dvmd_tls.o)
                              d:/ahl-gec-ide(4.26)º¬python/gcc/bin/../lib/gcc/arm-none-eabi/7.2.1/thumb/v7e-m/fpv4-sp/hard\libgcc.a(_aeabi_uldivmod.o) (__aeabi_ldiv0)
d:/ahl-gec-ide(4.26)º¬python/gcc/bin/../lib/gcc/arm-none-eabi/7.2.1/../../../../arm-none-eabi/lib/thumb/v7e-m/fpv4-sp/hard\libnosys.a(_exit.o)
                              d:/ahl-gec-ide(4.26)º¬python/gcc/bin/../lib/gcc/arm-none-eabi/7.2.1/../../../../arm-none-eabi/lib/thumb/v7e-m/fpv4-sp/hard\libc_nano.a(lib_a-exit.o) (_exit)

Allocating common symbols
Common symbol       size              file

component_fun       0x4               ./obj/startup_msp432p401r_gcc.o
gcRecvLen           0x2               ./obj/main.o
gcRecvDCLen         0x2               ./obj/main.o
gcRecvBuf           0x1000            ./obj/main.o

Discarded input sections

 .fini_array    0x00000000        0x4 d:/ahl-gec-ide(4.26)º¬python/gcc/bin/../lib/gcc/arm-none-eabi/7.2.1/thumb/v7e-m/fpv4-sp/hard/crtbegin.o
 .ARM.extab     0x00000000        0x0 d:/ahl-gec-ide(4.26)º¬python/gcc/bin/../lib/gcc/arm-none-eabi/7.2.1/../../../../arm-none-eabi/lib/thumb/v7e-m/fpv4-sp/hard/crt0.o
 .ARM.extab     0x00000000        0x0 d:/ahl-gec-ide(4.26)º¬python/gcc/bin/../lib/gcc/arm-none-eabi/7.2.1/thumb/v7e-m/fpv4-sp/hard\libgcc.a(_udivmoddi4.o)
 .eh_frame      0x00000000        0x4 d:/ahl-gec-ide(4.26)º¬python/gcc/bin/../lib/gcc/arm-none-eabi/7.2.1/thumb/v7e-m/fpv4-sp/hard/crtend.o
 .init          0x00000000        0x8 d:/ahl-gec-ide(4.26)º¬python/gcc/bin/../lib/gcc/arm-none-eabi/7.2.1/thumb/v7e-m/fpv4-sp/hard/crtn.o
 .fini          0x00000000        0x8 d:/ahl-gec-ide(4.26)º¬python/gcc/bin/../lib/gcc/arm-none-eabi/7.2.1/thumb/v7e-m/fpv4-sp/hard/crtn.o

Memory Configuration

Name             Origin             Length             Attributes
USER_INTVEC      0x0001a000         0x00001000         xr
MAIN_FLASH       0x0001b000         0x00025000         xr
SRAM_DATA        0x20002000         0x0000e000         rw
*default*        0x00000000         0xffffffff

Linker script and memory map

LOAD d:/ahl-gec-ide(4.26)º¬python/gcc/bin/../lib/gcc/arm-none-eabi/7.2.1/thumb/v7e-m/fpv4-sp/hard/crti.o
LOAD d:/ahl-gec-ide(4.26)º¬python/gcc/bin/../lib/gcc/arm-none-eabi/7.2.1/thumb/v7e-m/fpv4-sp/hard/crtbegin.o
LOAD d:/ahl-gec-ide(4.26)º¬python/gcc/bin/../lib/gcc/arm-none-eabi/7.2.1/../../../../arm-none-eabi/lib/thumb/v7e-m/fpv4-sp/hard/crt0.o
LOAD ./obj/emuart.o
LOAD ./obj/system_msp432p401r.o
LOAD ./obj/startup_msp432p401r_gcc.o
LOAD ./obj/main.o
LOAD ./obj/flash.o
LOAD ./obj/gpio.o
LOAD ./obj/gec.o
LOAD ./obj/uart.o
LOAD ./obj/isr.o
LOAD ./obj/printf.o
START GROUP
LOAD d:/ahl-gec-ide(4.26)º¬python/gcc/bin/../lib/gcc/arm-none-eabi/7.2.1/../../../../arm-none-eabi/lib/thumb/v7e-m/fpv4-sp/hard\libc_nano.a
LOAD d:/ahl-gec-ide(4.26)º¬python/gcc/bin/../lib/gcc/arm-none-eabi/7.2.1/../../../../arm-none-eabi/lib/thumb/v7e-m/fpv4-sp/hard\libm.a
END GROUP
START GROUP
LOAD d:/ahl-gec-ide(4.26)º¬python/gcc/bin/../lib/gcc/arm-none-eabi/7.2.1/thumb/v7e-m/fpv4-sp/hard\libgcc.a
LOAD d:/ahl-gec-ide(4.26)º¬python/gcc/bin/../lib/gcc/arm-none-eabi/7.2.1/../../../../arm-none-eabi/lib/thumb/v7e-m/fpv4-sp/hard\libc_nano.a
END GROUP
START GROUP
LOAD d:/ahl-gec-ide(4.26)º¬python/gcc/bin/../lib/gcc/arm-none-eabi/7.2.1/thumb/v7e-m/fpv4-sp/hard\libgcc.a
LOAD d:/ahl-gec-ide(4.26)º¬python/gcc/bin/../lib/gcc/arm-none-eabi/7.2.1/../../../../arm-none-eabi/lib/thumb/v7e-m/fpv4-sp/hard\libc_nano.a
LOAD d:/ahl-gec-ide(4.26)º¬python/gcc/bin/../lib/gcc/arm-none-eabi/7.2.1/../../../../arm-none-eabi/lib/thumb/v7e-m/fpv4-sp/hard\libnosys.a
END GROUP
START GROUP
LOAD d:/ahl-gec-ide(4.26)º¬python/gcc/bin/../lib/gcc/arm-none-eabi/7.2.1/thumb/v7e-m/fpv4-sp/hard\libgcc.a
LOAD d:/ahl-gec-ide(4.26)º¬python/gcc/bin/../lib/gcc/arm-none-eabi/7.2.1/../../../../arm-none-eabi/lib/thumb/v7e-m/fpv4-sp/hard\libc_nano.a
LOAD d:/ahl-gec-ide(4.26)º¬python/gcc/bin/../lib/gcc/arm-none-eabi/7.2.1/../../../../arm-none-eabi/lib/thumb/v7e-m/fpv4-sp/hard\libnosys.a
END GROUP
LOAD d:/ahl-gec-ide(4.26)º¬python/gcc/bin/../lib/gcc/arm-none-eabi/7.2.1/thumb/v7e-m/fpv4-sp/hard/crtend.o
LOAD d:/ahl-gec-ide(4.26)º¬python/gcc/bin/../lib/gcc/arm-none-eabi/7.2.1/thumb/v7e-m/fpv4-sp/hard/crtn.o
                0x00001000                MCU_SECTORSIZE = 0x1000
                0x00000000                MCU_FLASH_ADDR_START = 0x0
                0x0000001a                GEC_USER_SECTOR_START = 0x1a
                0x0000003f                GEC_USER_SECTOR_END = 0x3f
                0x20002000                GEC_USER_RAM_START = 0x20002000
                0x20010000                GEC_USER_RAM_END = 0x20010000
                0x0001a000                PROVIDE (_intvecs_base_address, DEFINED (_intvecs_base_address)?_intvecs_base_address:(MCU_SECTORSIZE * GEC_USER_SECTOR_START))

.intvecs        0x0001a000       0xe4
 *(.intvecs)
 .intvecs       0x0001a000       0xe4 ./obj/startup_msp432p401r_gcc.o
                0x0001a000                interruptVectors
                0x20002000                PROVIDE (_vtable_base_address, DEFINED (_vtable_base_address)?_vtable_base_address:GEC_USER_RAM_START)

.vtable
 *(.vtable)

.text           0x0001b000     0x477c
 CREATE_OBJECT_SYMBOLS
 *(.text)
 .text          0x0001b000        0x0 d:/ahl-gec-ide(4.26)º¬python/gcc/bin/../lib/gcc/arm-none-eabi/7.2.1/thumb/v7e-m/fpv4-sp/hard/crti.o
 .text          0x0001b000       0x40 d:/ahl-gec-ide(4.26)º¬python/gcc/bin/../lib/gcc/arm-none-eabi/7.2.1/thumb/v7e-m/fpv4-sp/hard/crtbegin.o
 .text          0x0001b040       0x74 d:/ahl-gec-ide(4.26)º¬python/gcc/bin/../lib/gcc/arm-none-eabi/7.2.1/../../../../arm-none-eabi/lib/thumb/v7e-m/fpv4-sp/hard/crt0.o
                0x0001b040                _start
                0x0001b040                _mainCRTStartup
 .text          0x0001b0b4      0x6e8 ./obj/emuart.o
                0x0001b0b4                emuart_init
                0x0001b0e4                emuart_send1
                0x0001b100                emuart_sendN
                0x0001b11e                emuart_send_string
                0x0001b150                emuart_frame
                0x0001b3c4                useremuart_frame
                0x0001b660                sendFrame
                0x0001b724                crc16
 .text          0x0001b79c      0x3c8 ./obj/system_msp432p401r.o
                0x0001b79c                SystemCoreClockUpdate
                0x0001ba9c                SystemInit
 .text          0x0001bb64       0x6c ./obj/startup_msp432p401r_gcc.o
                0x0001bb64                Reset_Handler
                0x0001bbc0                DebugMon_Handler
                0x0001bbc0                AES256_IRQHandler
                0x0001bbc0                HardFault_Handler
                0x0001bbc0                SysTick_Handler
                0x0001bbc0                PendSV_Handler
                0x0001bbc0                NMI_Handler
                0x0001bbc0                RTC_C_IRQHandler
                0x0001bbc0                PORT1_IRQHandler
                0x0001bbc0                FPU_IRQHandler
                0x0001bbc0                PORT2_IRQHandler
                0x0001bbc0                TA3_0_IRQHandler
                0x0001bbc0                UsageFault_Handler
                0x0001bbc0                DMA_INT3_IRQHandler
                0x0001bbc0                TA2_0_IRQHandler
                0x0001bbc0                DMA_INT1_IRQHandler
                0x0001bbc0                WDT_A_IRQHandler
                0x0001bbc0                TA2_N_IRQHandler
                0x0001bbc0                TA1_0_IRQHandler
                0x0001bbc0                CS_IRQHandler
                0x0001bbc0                PSS_IRQHandler
                0x0001bbc0                DMA_INT2_IRQHandler
                0x0001bbc0                DMA_INT0_IRQHandler
                0x0001bbc0                PORT4_IRQHandler
                0x0001bbc0                PORT5_IRQHandler
                0x0001bbc0                EUSCIB0_IRQHandler
                0x0001bbc0                Default_Handler
                0x0001bbc0                T32_INTC_IRQHandler
                0x0001bbc0                TA3_N_IRQHandler
                0x0001bbc0                TA0_0_IRQHandler
                0x0001bbc0                EUSCIA2_IRQHandler
                0x0001bbc0                PORT6_IRQHandler
                0x0001bbc0                PORT3_IRQHandler
                0x0001bbc0                MemManage_Handler
                0x0001bbc0                SVC_Handler
                0x0001bbc0                TA1_N_IRQHandler
                0x0001bbc0                EUSCIA1_IRQHandler
                0x0001bbc0                COMP_E1_IRQHandler
                0x0001bbc0                EUSCIB2_IRQHandler
                0x0001bbc0                FLCTL_IRQHandler
                0x0001bbc0                EUSCIB3_IRQHandler
                0x0001bbc0                T32_INT1_IRQHandler
                0x0001bbc0                DMA_ERR_IRQHandler
                0x0001bbc0                ADC14_IRQHandler
                0x0001bbc0                EUSCIA0_IRQHandler
                0x0001bbc0                BusFault_Handler
                0x0001bbc0                PCM_IRQHandler
                0x0001bbc0                TA0_N_IRQHandler
                0x0001bbc0                COMP_E0_IRQHandler
                0x0001bbc0                EUSCIB1_IRQHandler
                0x0001bbc0                T32_INT2_IRQHandler
 .text          0x0001bbd0       0x98 ./obj/main.o
                0x0001bbd0                main
 .text          0x0001bc68      0x830 ./obj/flash.o
                0x0001bc68                flash_init
                0x0001bc94                flash_erase
                0x0001bde8                flash_write
                0x0001bf94                flash_write_physical
                0x0001c118                flash_read_physical
                0x0001c13e                flash_read_logic
                0x0001c1e6                flash_protect
                0x0001c2a0                flash_unprotect
                0x0001c360                flash_isSectorProtected
                0x0001c3e0                flash_isempty
 .text          0x0001c498      0xc58 ./obj/gpio.o
                0x0001c52e                gpio_init
                0x0001c800                gpio_set
                0x0001c940                gpio_get
                0x0001ca00                gpio_reverse
                0x0001cb68                gpio_pull
                0x0001cca8                gpio_enable_int
                0x0001ce60                gpio_disable_int
                0x0001cf50                gpio_drive_strength
 .text          0x0001d0f0      0x394 ./obj/gec.o
                0x0001d118                Vectors_Init
                0x0001d1ec                SYSTEM_FUNCTION
 *fill*         0x0001d484        0x4 
 .text          0x0001d488      0x640 ./obj/uart.o
                0x0001d4f0                uart_init
                0x0001d710                uart_send1
                0x0001d788                uart_sendN
                0x0001d7f0                uart_send_string
                0x0001d854                uart_re1
                0x0001d8d8                uart_reN
                0x0001d946                uart_enable_re_int
                0x0001d998                uart_disable_re_int
                0x0001d9e8                uart_get_re_int
                0x0001da38                uart_is_uartNo
                0x0001da5a                BRSxSel
 .text          0x0001dac8       0xcc ./obj/isr.o
                0x0001dac8                EUSCIA3_IRQHandler
                0x0001db16                User_SysFun
 *fill*         0x0001db94        0x4 
 .text          0x0001db98      0xec4 ./obj/printf.o
                0x0001db98                out_char
                0x0001dc04                printk_mkfloatstr
                0x0001e082                printk
                0x0001ea20                myprintf
 .text          0x0001ea5c        0x0 d:/ahl-gec-ide(4.26)º¬python/gcc/bin/../lib/gcc/arm-none-eabi/7.2.1/../../../../arm-none-eabi/lib/thumb/v7e-m/fpv4-sp/hard\libc_nano.a(lib_a-exit.o)
 .text          0x0001ea5c        0x0 d:/ahl-gec-ide(4.26)º¬python/gcc/bin/../lib/gcc/arm-none-eabi/7.2.1/../../../../arm-none-eabi/lib/thumb/v7e-m/fpv4-sp/hard\libc_nano.a(lib_a-impure.o)
 .text          0x0001ea5c        0x0 d:/ahl-gec-ide(4.26)º¬python/gcc/bin/../lib/gcc/arm-none-eabi/7.2.1/../../../../arm-none-eabi/lib/thumb/v7e-m/fpv4-sp/hard\libc_nano.a(lib_a-init.o)
 .text          0x0001ea5c        0x0 d:/ahl-gec-ide(4.26)º¬python/gcc/bin/../lib/gcc/arm-none-eabi/7.2.1/../../../../arm-none-eabi/lib/thumb/v7e-m/fpv4-sp/hard\libc_nano.a(lib_a-memcpy-stub.o)
 .text          0x0001ea5c        0x0 d:/ahl-gec-ide(4.26)º¬python/gcc/bin/../lib/gcc/arm-none-eabi/7.2.1/../../../../arm-none-eabi/lib/thumb/v7e-m/fpv4-sp/hard\libc_nano.a(lib_a-memset.o)
 .text          0x0001ea5c       0x14 d:/ahl-gec-ide(4.26)º¬python/gcc/bin/../lib/gcc/arm-none-eabi/7.2.1/../../../../arm-none-eabi/lib/thumb/v7e-m/fpv4-sp/hard\libc_nano.a(lib_a-strcmp.o)
                0x0001ea5c                strcmp
 .text          0x0001ea70       0x10 d:/ahl-gec-ide(4.26)º¬python/gcc/bin/../lib/gcc/arm-none-eabi/7.2.1/../../../../arm-none-eabi/lib/thumb/v7e-m/fpv4-sp/hard\libc_nano.a(lib_a-strlen.o)
                0x0001ea70                strlen
 .text          0x0001ea80        0x0 d:/ahl-gec-ide(4.26)º¬python/gcc/bin/../lib/gcc/arm-none-eabi/7.2.1/../../../../arm-none-eabi/lib/thumb/v7e-m/fpv4-sp/hard\libc_nano.a(lib_a-strncmp.o)
 .text          0x0001ea80      0x378 d:/ahl-gec-ide(4.26)º¬python/gcc/bin/../lib/gcc/arm-none-eabi/7.2.1/thumb/v7e-m/fpv4-sp/hard\libgcc.a(_arm_addsubdf3.o)
                0x0001ea80                __aeabi_drsub
                0x0001ea88                __aeabi_dsub
                0x0001ea88                __subdf3
                0x0001ea8c                __aeabi_dadd
                0x0001ea8c                __adddf3
                0x0001ed04                __floatunsidf
                0x0001ed04                __aeabi_ui2d
                0x0001ed24                __floatsidf
                0x0001ed24                __aeabi_i2d
                0x0001ed48                __aeabi_f2d
                0x0001ed48                __extendsfdf2
                0x0001ed8c                __floatundidf
                0x0001ed8c                __aeabi_ul2d
                0x0001ed9c                __floatdidf
                0x0001ed9c                __aeabi_l2d
 .text          0x0001edf8      0x424 d:/ahl-gec-ide(4.26)º¬python/gcc/bin/../lib/gcc/arm-none-eabi/7.2.1/thumb/v7e-m/fpv4-sp/hard\libgcc.a(_arm_muldivdf3.o)
                0x0001edf8                __aeabi_dmul
                0x0001edf8                __muldf3
                0x0001f04c                __divdf3
                0x0001f04c                __aeabi_ddiv
 .text          0x0001f21c      0x110 d:/ahl-gec-ide(4.26)º¬python/gcc/bin/../lib/gcc/arm-none-eabi/7.2.1/thumb/v7e-m/fpv4-sp/hard\libgcc.a(_arm_cmpdf2.o)
                0x0001f21c                __gtdf2
                0x0001f21c                __gedf2
                0x0001f224                __ltdf2
                0x0001f224                __ledf2
                0x0001f22c                __nedf2
                0x0001f22c                __eqdf2
                0x0001f22c                __cmpdf2
                0x0001f2a8                __aeabi_cdrcmple
                0x0001f2b8                __aeabi_cdcmpeq
                0x0001f2b8                __aeabi_cdcmple
                0x0001f2c8                __aeabi_dcmpeq
                0x0001f2dc                __aeabi_dcmplt
                0x0001f2f0                __aeabi_dcmple
                0x0001f304                __aeabi_dcmpge
                0x0001f318                __aeabi_dcmpgt
 .text          0x0001f32c       0x40 d:/ahl-gec-ide(4.26)º¬python/gcc/bin/../lib/gcc/arm-none-eabi/7.2.1/thumb/v7e-m/fpv4-sp/hard\libgcc.a(_arm_fixunsdfsi.o)
                0x0001f32c                __aeabi_d2uiz
                0x0001f32c                __fixunsdfsi
 .text          0x0001f36c       0x30 d:/ahl-gec-ide(4.26)º¬python/gcc/bin/../lib/gcc/arm-none-eabi/7.2.1/thumb/v7e-m/fpv4-sp/hard\libgcc.a(_aeabi_uldivmod.o)
                0x0001f36c                __aeabi_uldivmod
 .text          0x0001f39c       0x44 d:/ahl-gec-ide(4.26)º¬python/gcc/bin/../lib/gcc/arm-none-eabi/7.2.1/thumb/v7e-m/fpv4-sp/hard\libgcc.a(_fixunsdfdi.o)
                0x0001f39c                __fixunsdfdi
                0x0001f39c                __aeabi_d2ulz
 .text          0x0001f3e0      0x2cc d:/ahl-gec-ide(4.26)º¬python/gcc/bin/../lib/gcc/arm-none-eabi/7.2.1/thumb/v7e-m/fpv4-sp/hard\libgcc.a(_udivmoddi4.o)
                0x0001f3e0                __udivmoddi4
 .text          0x0001f6ac        0x4 d:/ahl-gec-ide(4.26)º¬python/gcc/bin/../lib/gcc/arm-none-eabi/7.2.1/thumb/v7e-m/fpv4-sp/hard\libgcc.a(_dvmd_tls.o)
                0x0001f6ac                __aeabi_idiv0
                0x0001f6ac                __aeabi_ldiv0
 .text          0x0001f6b0        0x0 d:/ahl-gec-ide(4.26)º¬python/gcc/bin/../lib/gcc/arm-none-eabi/7.2.1/../../../../arm-none-eabi/lib/thumb/v7e-m/fpv4-sp/hard\libnosys.a(_exit.o)
 .text          0x0001f6b0        0x0 d:/ahl-gec-ide(4.26)º¬python/gcc/bin/../lib/gcc/arm-none-eabi/7.2.1/thumb/v7e-m/fpv4-sp/hard/crtend.o
 .text          0x0001f6b0        0x0 d:/ahl-gec-ide(4.26)º¬python/gcc/bin/../lib/gcc/arm-none-eabi/7.2.1/thumb/v7e-m/fpv4-sp/hard/crtn.o
 *(.text.*)
 .text.exit     0x0001f6b0       0x28 d:/ahl-gec-ide(4.26)º¬python/gcc/bin/../lib/gcc/arm-none-eabi/7.2.1/../../../../arm-none-eabi/lib/thumb/v7e-m/fpv4-sp/hard\libc_nano.a(lib_a-exit.o)
                0x0001f6b0                exit
 .text.__libc_init_array
                0x0001f6d8       0x48 d:/ahl-gec-ide(4.26)º¬python/gcc/bin/../lib/gcc/arm-none-eabi/7.2.1/../../../../arm-none-eabi/lib/thumb/v7e-m/fpv4-sp/hard\libc_nano.a(lib_a-init.o)
                0x0001f6d8                __libc_init_array
 .text.memcpy   0x0001f720       0x16 d:/ahl-gec-ide(4.26)º¬python/gcc/bin/../lib/gcc/arm-none-eabi/7.2.1/../../../../arm-none-eabi/lib/thumb/v7e-m/fpv4-sp/hard\libc_nano.a(lib_a-memcpy-stub.o)
                0x0001f720                memcpy
 .text.memset   0x0001f736       0x10 d:/ahl-gec-ide(4.26)º¬python/gcc/bin/../lib/gcc/arm-none-eabi/7.2.1/../../../../arm-none-eabi/lib/thumb/v7e-m/fpv4-sp/hard\libc_nano.a(lib_a-memset.o)
                0x0001f736                memset
 .text.strncmp  0x0001f746       0x24 d:/ahl-gec-ide(4.26)º¬python/gcc/bin/../lib/gcc/arm-none-eabi/7.2.1/../../../../arm-none-eabi/lib/thumb/v7e-m/fpv4-sp/hard\libc_nano.a(lib_a-strncmp.o)
                0x0001f746                strncmp
 *fill*         0x0001f76a        0x2 
 .text._exit    0x0001f76c        0x4 d:/ahl-gec-ide(4.26)º¬python/gcc/bin/../lib/gcc/arm-none-eabi/7.2.1/../../../../arm-none-eabi/lib/thumb/v7e-m/fpv4-sp/hard\libnosys.a(_exit.o)
                0x0001f76c                _exit
                0x0001f770                . = ALIGN (0x4)
 *(.ctors)
                0x0001f770                . = ALIGN (0x4)
 *(.dtors)
                0x0001f770                . = ALIGN (0x4)
                0x0001f770                __init_array_start = .
 *(.init_array*)
 .init_array    0x0001f770        0x4 d:/ahl-gec-ide(4.26)º¬python/gcc/bin/../lib/gcc/arm-none-eabi/7.2.1/thumb/v7e-m/fpv4-sp/hard/crtbegin.o
                0x0001f774                __init_array_end = .
 *(.init)
 .init          0x0001f774        0x4 d:/ahl-gec-ide(4.26)º¬python/gcc/bin/../lib/gcc/arm-none-eabi/7.2.1/thumb/v7e-m/fpv4-sp/hard/crti.o
                0x0001f774                _init
 *(.fini*)
 .fini          0x0001f778        0x4 d:/ahl-gec-ide(4.26)º¬python/gcc/bin/../lib/gcc/arm-none-eabi/7.2.1/thumb/v7e-m/fpv4-sp/hard/crti.o
                0x0001f778                _fini

.glue_7         0x0001f77c        0x0
 .glue_7        0x0001f77c        0x0 linker stubs

.glue_7t        0x0001f77c        0x0
 .glue_7t       0x0001f77c        0x0 linker stubs

.vfp11_veneer   0x0001f77c        0x0
 .vfp11_veneer  0x0001f77c        0x0 linker stubs

.v4_bx          0x0001f77c        0x0
 .v4_bx         0x0001f77c        0x0 linker stubs

.iplt           0x0001f77c        0x0
 .iplt          0x0001f77c        0x0 d:/ahl-gec-ide(4.26)º¬python/gcc/bin/../lib/gcc/arm-none-eabi/7.2.1/thumb/v7e-m/fpv4-sp/hard/crtbegin.o

.rodata         0x0001f77c      0x100
 *(.rodata)
 .rodata        0x0001f77c       0x2f ./obj/emuart.o
 *fill*         0x0001f7ab        0x1 
 .rodata        0x0001f7ac       0x47 ./obj/main.o
 *fill*         0x0001f7f3        0x1 
 .rodata        0x0001f7f4       0x7f ./obj/gec.o
 *fill*         0x0001f873        0x1 
 .rodata        0x0001f874        0x4 ./obj/uart.o
 *(.rodata.*)
 .rodata._global_impure_ptr
                0x0001f878        0x4 d:/ahl-gec-ide(4.26)º¬python/gcc/bin/../lib/gcc/arm-none-eabi/7.2.1/../../../../arm-none-eabi/lib/thumb/v7e-m/fpv4-sp/hard\libc_nano.a(lib_a-impure.o)
                0x0001f878                _global_impure_ptr

.eh_frame       0x0001f87c        0x0
 .eh_frame      0x0001f87c        0x0 d:/ahl-gec-ide(4.26)º¬python/gcc/bin/../lib/gcc/arm-none-eabi/7.2.1/thumb/v7e-m/fpv4-sp/hard/crtbegin.o

.ARM.exidx      0x0001f87c        0x8
                0x0001f87c                __exidx_start = .
 *(.ARM.exidx* .gnu.linkonce.armexidx.*)
 .ARM.exidx     0x0001f87c        0x8 d:/ahl-gec-ide(4.26)º¬python/gcc/bin/../lib/gcc/arm-none-eabi/7.2.1/../../../../arm-none-eabi/lib/thumb/v7e-m/fpv4-sp/hard/crt0.o
 .ARM.exidx     0x0001f884        0x0 d:/ahl-gec-ide(4.26)º¬python/gcc/bin/../lib/gcc/arm-none-eabi/7.2.1/thumb/v7e-m/fpv4-sp/hard\libgcc.a(_udivmoddi4.o)
                                  0x8 (size before relaxing)
                0x0001f884                __exidx_end = .

.rel.dyn        0x0001f884        0x0
 .rel.iplt      0x0001f884        0x0 d:/ahl-gec-ide(4.26)º¬python/gcc/bin/../lib/gcc/arm-none-eabi/7.2.1/thumb/v7e-m/fpv4-sp/hard/crtbegin.o

.ARM.extab
 *(.ARM.extab* .gnu.linkonce.armextab.*)
                0x0001f884                __etext = .

.data           0x20002000      0x134 load address 0x0001f884
                0x0001f884                __data_load__ = LOADADDR (.data)
                0x20002000                __data_start__ = .
 *(.data)
 .data          0x20002000        0x0 d:/ahl-gec-ide(4.26)º¬python/gcc/bin/../lib/gcc/arm-none-eabi/7.2.1/thumb/v7e-m/fpv4-sp/hard/crti.o
 .data          0x20002000        0x4 d:/ahl-gec-ide(4.26)º¬python/gcc/bin/../lib/gcc/arm-none-eabi/7.2.1/thumb/v7e-m/fpv4-sp/hard/crtbegin.o
                0x20002000                __dso_handle
 .data          0x20002004        0x0 d:/ahl-gec-ide(4.26)º¬python/gcc/bin/../lib/gcc/arm-none-eabi/7.2.1/../../../../arm-none-eabi/lib/thumb/v7e-m/fpv4-sp/hard/crt0.o
 .data          0x20002004       0x24 ./obj/emuart.o
 .data          0x20002028        0x4 ./obj/system_msp432p401r.o
                0x20002028                SystemCoreClock
 .data          0x2000202c        0x0 ./obj/startup_msp432p401r_gcc.o
 .data          0x2000202c        0x0 ./obj/main.o
 .data          0x2000202c        0x0 ./obj/flash.o
 .data          0x2000202c       0x28 ./obj/gpio.o
                0x2000202c                GPIO_ODD_ARR
                0x20002040                GPIO_EVEN_ARR
 .data          0x20002054        0x0 ./obj/gec.o
 .data          0x20002054       0x7c ./obj/uart.o
                0x20002064                BRSxS
                0x200020ac                ValBRSxS
 .data          0x200020d0        0x0 ./obj/isr.o
 .data          0x200020d0        0x0 ./obj/printf.o
 .data          0x200020d0        0x0 d:/ahl-gec-ide(4.26)º¬python/gcc/bin/../lib/gcc/arm-none-eabi/7.2.1/../../../../arm-none-eabi/lib/thumb/v7e-m/fpv4-sp/hard\libc_nano.a(lib_a-exit.o)
 .data          0x200020d0        0x0 d:/ahl-gec-ide(4.26)º¬python/gcc/bin/../lib/gcc/arm-none-eabi/7.2.1/../../../../arm-none-eabi/lib/thumb/v7e-m/fpv4-sp/hard\libc_nano.a(lib_a-impure.o)
 .data          0x200020d0        0x0 d:/ahl-gec-ide(4.26)º¬python/gcc/bin/../lib/gcc/arm-none-eabi/7.2.1/../../../../arm-none-eabi/lib/thumb/v7e-m/fpv4-sp/hard\libc_nano.a(lib_a-init.o)
 .data          0x200020d0        0x0 d:/ahl-gec-ide(4.26)º¬python/gcc/bin/../lib/gcc/arm-none-eabi/7.2.1/../../../../arm-none-eabi/lib/thumb/v7e-m/fpv4-sp/hard\libc_nano.a(lib_a-memcpy-stub.o)
 .data          0x200020d0        0x0 d:/ahl-gec-ide(4.26)º¬python/gcc/bin/../lib/gcc/arm-none-eabi/7.2.1/../../../../arm-none-eabi/lib/thumb/v7e-m/fpv4-sp/hard\libc_nano.a(lib_a-memset.o)
 .data          0x200020d0        0x0 d:/ahl-gec-ide(4.26)º¬python/gcc/bin/../lib/gcc/arm-none-eabi/7.2.1/../../../../arm-none-eabi/lib/thumb/v7e-m/fpv4-sp/hard\libc_nano.a(lib_a-strcmp.o)
 .data          0x200020d0        0x0 d:/ahl-gec-ide(4.26)º¬python/gcc/bin/../lib/gcc/arm-none-eabi/7.2.1/../../../../arm-none-eabi/lib/thumb/v7e-m/fpv4-sp/hard\libc_nano.a(lib_a-strlen.o)
 .data          0x200020d0        0x0 d:/ahl-gec-ide(4.26)º¬python/gcc/bin/../lib/gcc/arm-none-eabi/7.2.1/../../../../arm-none-eabi/lib/thumb/v7e-m/fpv4-sp/hard\libc_nano.a(lib_a-strncmp.o)
 .data          0x200020d0        0x0 d:/ahl-gec-ide(4.26)º¬python/gcc/bin/../lib/gcc/arm-none-eabi/7.2.1/thumb/v7e-m/fpv4-sp/hard\libgcc.a(_arm_addsubdf3.o)
 .data          0x200020d0        0x0 d:/ahl-gec-ide(4.26)º¬python/gcc/bin/../lib/gcc/arm-none-eabi/7.2.1/thumb/v7e-m/fpv4-sp/hard\libgcc.a(_arm_muldivdf3.o)
 .data          0x200020d0        0x0 d:/ahl-gec-ide(4.26)º¬python/gcc/bin/../lib/gcc/arm-none-eabi/7.2.1/thumb/v7e-m/fpv4-sp/hard\libgcc.a(_arm_cmpdf2.o)
 .data          0x200020d0        0x0 d:/ahl-gec-ide(4.26)º¬python/gcc/bin/../lib/gcc/arm-none-eabi/7.2.1/thumb/v7e-m/fpv4-sp/hard\libgcc.a(_arm_fixunsdfsi.o)
 .data          0x200020d0        0x0 d:/ahl-gec-ide(4.26)º¬python/gcc/bin/../lib/gcc/arm-none-eabi/7.2.1/thumb/v7e-m/fpv4-sp/hard\libgcc.a(_aeabi_uldivmod.o)
 .data          0x200020d0        0x0 d:/ahl-gec-ide(4.26)º¬python/gcc/bin/../lib/gcc/arm-none-eabi/7.2.1/thumb/v7e-m/fpv4-sp/hard\libgcc.a(_fixunsdfdi.o)
 .data          0x200020d0        0x0 d:/ahl-gec-ide(4.26)º¬python/gcc/bin/../lib/gcc/arm-none-eabi/7.2.1/thumb/v7e-m/fpv4-sp/hard\libgcc.a(_udivmoddi4.o)
 .data          0x200020d0        0x0 d:/ahl-gec-ide(4.26)º¬python/gcc/bin/../lib/gcc/arm-none-eabi/7.2.1/thumb/v7e-m/fpv4-sp/hard\libgcc.a(_dvmd_tls.o)
 .data          0x200020d0        0x0 d:/ahl-gec-ide(4.26)º¬python/gcc/bin/../lib/gcc/arm-none-eabi/7.2.1/../../../../arm-none-eabi/lib/thumb/v7e-m/fpv4-sp/hard\libnosys.a(_exit.o)
 .data          0x200020d0        0x0 d:/ahl-gec-ide(4.26)º¬python/gcc/bin/../lib/gcc/arm-none-eabi/7.2.1/thumb/v7e-m/fpv4-sp/hard/crtend.o
 .data          0x200020d0        0x0 d:/ahl-gec-ide(4.26)º¬python/gcc/bin/../lib/gcc/arm-none-eabi/7.2.1/thumb/v7e-m/fpv4-sp/hard/crtn.o
 *(.data*)
 .data._impure_ptr
                0x200020d0        0x4 d:/ahl-gec-ide(4.26)º¬python/gcc/bin/../lib/gcc/arm-none-eabi/7.2.1/../../../../arm-none-eabi/lib/thumb/v7e-m/fpv4-sp/hard\libc_nano.a(lib_a-impure.o)
                0x200020d0                _impure_ptr
 .data.impure_data
                0x200020d4       0x60 d:/ahl-gec-ide(4.26)º¬python/gcc/bin/../lib/gcc/arm-none-eabi/7.2.1/../../../../arm-none-eabi/lib/thumb/v7e-m/fpv4-sp/hard\libc_nano.a(lib_a-impure.o)
                0x20002134                . = ALIGN (0x4)
                0x20002134                __data_end__ = .

.igot.plt       0x20002134        0x0 load address 0x0001f9b8
 .igot.plt      0x20002134        0x0 d:/ahl-gec-ide(4.26)º¬python/gcc/bin/../lib/gcc/arm-none-eabi/7.2.1/thumb/v7e-m/fpv4-sp/hard/crtbegin.o

.bss            0x20002134     0x1028
                0x20002134                __bss_start__ = .
 *(.shbss)
 *(.bss)
 .bss           0x20002134        0x0 d:/ahl-gec-ide(4.26)º¬python/gcc/bin/../lib/gcc/arm-none-eabi/7.2.1/thumb/v7e-m/fpv4-sp/hard/crti.o
 .bss           0x20002134       0x1c d:/ahl-gec-ide(4.26)º¬python/gcc/bin/../lib/gcc/arm-none-eabi/7.2.1/thumb/v7e-m/fpv4-sp/hard/crtbegin.o
 .bss           0x20002150        0x0 d:/ahl-gec-ide(4.26)º¬python/gcc/bin/../lib/gcc/arm-none-eabi/7.2.1/../../../../arm-none-eabi/lib/thumb/v7e-m/fpv4-sp/hard/crt0.o
 .bss           0x20002150        0x1 ./obj/emuart.o
 .bss           0x20002151        0x0 ./obj/system_msp432p401r.o
 .bss           0x20002151        0x0 ./obj/startup_msp432p401r_gcc.o
 .bss           0x20002151        0x0 ./obj/main.o
 .bss           0x20002151        0x0 ./obj/flash.o
 .bss           0x20002151        0x0 ./obj/gpio.o
 .bss           0x20002151        0x0 ./obj/gec.o
 .bss           0x20002151        0x0 ./obj/uart.o
 .bss           0x20002151        0x0 ./obj/isr.o
 .bss           0x20002151        0x0 ./obj/printf.o
 .bss           0x20002151        0x0 d:/ahl-gec-ide(4.26)º¬python/gcc/bin/../lib/gcc/arm-none-eabi/7.2.1/../../../../arm-none-eabi/lib/thumb/v7e-m/fpv4-sp/hard\libc_nano.a(lib_a-exit.o)
 .bss           0x20002151        0x0 d:/ahl-gec-ide(4.26)º¬python/gcc/bin/../lib/gcc/arm-none-eabi/7.2.1/../../../../arm-none-eabi/lib/thumb/v7e-m/fpv4-sp/hard\libc_nano.a(lib_a-impure.o)
 .bss           0x20002151        0x0 d:/ahl-gec-ide(4.26)º¬python/gcc/bin/../lib/gcc/arm-none-eabi/7.2.1/../../../../arm-none-eabi/lib/thumb/v7e-m/fpv4-sp/hard\libc_nano.a(lib_a-init.o)
 .bss           0x20002151        0x0 d:/ahl-gec-ide(4.26)º¬python/gcc/bin/../lib/gcc/arm-none-eabi/7.2.1/../../../../arm-none-eabi/lib/thumb/v7e-m/fpv4-sp/hard\libc_nano.a(lib_a-memcpy-stub.o)
 .bss           0x20002151        0x0 d:/ahl-gec-ide(4.26)º¬python/gcc/bin/../lib/gcc/arm-none-eabi/7.2.1/../../../../arm-none-eabi/lib/thumb/v7e-m/fpv4-sp/hard\libc_nano.a(lib_a-memset.o)
 .bss           0x20002151        0x0 d:/ahl-gec-ide(4.26)º¬python/gcc/bin/../lib/gcc/arm-none-eabi/7.2.1/../../../../arm-none-eabi/lib/thumb/v7e-m/fpv4-sp/hard\libc_nano.a(lib_a-strcmp.o)
 .bss           0x20002151        0x0 d:/ahl-gec-ide(4.26)º¬python/gcc/bin/../lib/gcc/arm-none-eabi/7.2.1/../../../../arm-none-eabi/lib/thumb/v7e-m/fpv4-sp/hard\libc_nano.a(lib_a-strlen.o)
 .bss           0x20002151        0x0 d:/ahl-gec-ide(4.26)º¬python/gcc/bin/../lib/gcc/arm-none-eabi/7.2.1/../../../../arm-none-eabi/lib/thumb/v7e-m/fpv4-sp/hard\libc_nano.a(lib_a-strncmp.o)
 .bss           0x20002151        0x0 d:/ahl-gec-ide(4.26)º¬python/gcc/bin/../lib/gcc/arm-none-eabi/7.2.1/thumb/v7e-m/fpv4-sp/hard\libgcc.a(_arm_addsubdf3.o)
 .bss           0x20002151        0x0 d:/ahl-gec-ide(4.26)º¬python/gcc/bin/../lib/gcc/arm-none-eabi/7.2.1/thumb/v7e-m/fpv4-sp/hard\libgcc.a(_arm_muldivdf3.o)
 .bss           0x20002151        0x0 d:/ahl-gec-ide(4.26)º¬python/gcc/bin/../lib/gcc/arm-none-eabi/7.2.1/thumb/v7e-m/fpv4-sp/hard\libgcc.a(_arm_cmpdf2.o)
 .bss           0x20002151        0x0 d:/ahl-gec-ide(4.26)º¬python/gcc/bin/../lib/gcc/arm-none-eabi/7.2.1/thumb/v7e-m/fpv4-sp/hard\libgcc.a(_arm_fixunsdfsi.o)
 .bss           0x20002151        0x0 d:/ahl-gec-ide(4.26)º¬python/gcc/bin/../lib/gcc/arm-none-eabi/7.2.1/thumb/v7e-m/fpv4-sp/hard\libgcc.a(_aeabi_uldivmod.o)
 .bss           0x20002151        0x0 d:/ahl-gec-ide(4.26)º¬python/gcc/bin/../lib/gcc/arm-none-eabi/7.2.1/thumb/v7e-m/fpv4-sp/hard\libgcc.a(_fixunsdfdi.o)
 .bss           0x20002151        0x0 d:/ahl-gec-ide(4.26)º¬python/gcc/bin/../lib/gcc/arm-none-eabi/7.2.1/thumb/v7e-m/fpv4-sp/hard\libgcc.a(_udivmoddi4.o)
 .bss           0x20002151        0x0 d:/ahl-gec-ide(4.26)º¬python/gcc/bin/../lib/gcc/arm-none-eabi/7.2.1/thumb/v7e-m/fpv4-sp/hard\libgcc.a(_dvmd_tls.o)
 .bss           0x20002151        0x0 d:/ahl-gec-ide(4.26)º¬python/gcc/bin/../lib/gcc/arm-none-eabi/7.2.1/../../../../arm-none-eabi/lib/thumb/v7e-m/fpv4-sp/hard\libnosys.a(_exit.o)
 .bss           0x20002151        0x0 d:/ahl-gec-ide(4.26)º¬python/gcc/bin/../lib/gcc/arm-none-eabi/7.2.1/thumb/v7e-m/fpv4-sp/hard/crtend.o
 .bss           0x20002151        0x0 d:/ahl-gec-ide(4.26)º¬python/gcc/bin/../lib/gcc/arm-none-eabi/7.2.1/thumb/v7e-m/fpv4-sp/hard/crtn.o
 *(.bss.*)
 *(COMMON)
 *fill*         0x20002151        0x3 
 COMMON         0x20002154        0x4 ./obj/startup_msp432p401r_gcc.o
                0x20002154                component_fun
 COMMON         0x20002158     0x1004 ./obj/main.o
                0x20002158                gcRecvLen
                0x2000215a                gcRecvDCLen
                0x2000215c                gcRecvBuf
                0x2000315c                . = ALIGN (0x4)
                0x2000315c                __bss_end__ = .

.heap           0x2000315c        0x4
                0x20003160                . = ALIGN (0x8)
 *fill*         0x2000315c        0x4 
                0x20003160                __end__ = .
                [!provide]                PROVIDE (end, .)
                0x20003160                __HeapBase = .
                0x20003160                __HeapLimit = .

.stack          0x20003160        0x0
                0x20003160                . = ALIGN (0x8)
                0x20010000                __StackTop = (ORIGIN (SRAM_DATA) + LENGTH (SRAM_DATA))
OUTPUT(GPIO-Output-ComponentMSP432-20210330.out elf32-littlearm)

.ARM.attributes
                0x00000000       0x30
 .ARM.attributes
                0x00000000       0x22 d:/ahl-gec-ide(4.26)º¬python/gcc/bin/../lib/gcc/arm-none-eabi/7.2.1/thumb/v7e-m/fpv4-sp/hard/crti.o
 .ARM.attributes
                0x00000022       0x34 d:/ahl-gec-ide(4.26)º¬python/gcc/bin/../lib/gcc/arm-none-eabi/7.2.1/thumb/v7e-m/fpv4-sp/hard/crtbegin.o
 .ARM.attributes
                0x00000056       0x20 d:/ahl-gec-ide(4.26)º¬python/gcc/bin/../lib/gcc/arm-none-eabi/7.2.1/../../../../arm-none-eabi/lib/thumb/v7e-m/fpv4-sp/hard/crt0.o
 .ARM.attributes
                0x00000076       0x39 ./obj/emuart.o
 .ARM.attributes
                0x000000af       0x39 ./obj/system_msp432p401r.o
 .ARM.attributes
                0x000000e8       0x39 ./obj/startup_msp432p401r_gcc.o
 .ARM.attributes
                0x00000121       0x39 ./obj/main.o
 .ARM.attributes
                0x0000015a       0x39 ./obj/flash.o
 .ARM.attributes
                0x00000193       0x39 ./obj/gpio.o
 .ARM.attributes
                0x000001cc       0x39 ./obj/gec.o
 .ARM.attributes
                0x00000205       0x39 ./obj/uart.o
 .ARM.attributes
                0x0000023e       0x39 ./obj/isr.o
 .ARM.attributes
                0x00000277       0x39 ./obj/printf.o
 .ARM.attributes
                0x000002b0       0x34 d:/ahl-gec-ide(4.26)º¬python/gcc/bin/../lib/gcc/arm-none-eabi/7.2.1/../../../../arm-none-eabi/lib/thumb/v7e-m/fpv4-sp/hard\libc_nano.a(lib_a-exit.o)
 .ARM.attributes
                0x000002e4       0x34 d:/ahl-gec-ide(4.26)º¬python/gcc/bin/../lib/gcc/arm-none-eabi/7.2.1/../../../../arm-none-eabi/lib/thumb/v7e-m/fpv4-sp/hard\libc_nano.a(lib_a-impure.o)
 .ARM.attributes
                0x00000318       0x34 d:/ahl-gec-ide(4.26)º¬python/gcc/bin/../lib/gcc/arm-none-eabi/7.2.1/../../../../arm-none-eabi/lib/thumb/v7e-m/fpv4-sp/hard\libc_nano.a(lib_a-init.o)
 .ARM.attributes
                0x0000034c       0x34 d:/ahl-gec-ide(4.26)º¬python/gcc/bin/../lib/gcc/arm-none-eabi/7.2.1/../../../../arm-none-eabi/lib/thumb/v7e-m/fpv4-sp/hard\libc_nano.a(lib_a-memcpy-stub.o)
 .ARM.attributes
                0x00000380       0x34 d:/ahl-gec-ide(4.26)º¬python/gcc/bin/../lib/gcc/arm-none-eabi/7.2.1/../../../../arm-none-eabi/lib/thumb/v7e-m/fpv4-sp/hard\libc_nano.a(lib_a-memset.o)
 .ARM.attributes
                0x000003b4       0x20 d:/ahl-gec-ide(4.26)º¬python/gcc/bin/../lib/gcc/arm-none-eabi/7.2.1/../../../../arm-none-eabi/lib/thumb/v7e-m/fpv4-sp/hard\libc_nano.a(lib_a-strcmp.o)
 .ARM.attributes
                0x000003d4       0x1b d:/ahl-gec-ide(4.26)º¬python/gcc/bin/../lib/gcc/arm-none-eabi/7.2.1/../../../../arm-none-eabi/lib/thumb/v7e-m/fpv4-sp/hard\libc_nano.a(lib_a-strlen.o)
 .ARM.attributes
                0x000003ef       0x34 d:/ahl-gec-ide(4.26)º¬python/gcc/bin/../lib/gcc/arm-none-eabi/7.2.1/../../../../arm-none-eabi/lib/thumb/v7e-m/fpv4-sp/hard\libc_nano.a(lib_a-strncmp.o)
 .ARM.attributes
                0x00000423       0x22 d:/ahl-gec-ide(4.26)º¬python/gcc/bin/../lib/gcc/arm-none-eabi/7.2.1/thumb/v7e-m/fpv4-sp/hard\libgcc.a(_arm_addsubdf3.o)
 .ARM.attributes
                0x00000445       0x22 d:/ahl-gec-ide(4.26)º¬python/gcc/bin/../lib/gcc/arm-none-eabi/7.2.1/thumb/v7e-m/fpv4-sp/hard\libgcc.a(_arm_muldivdf3.o)
 .ARM.attributes
                0x00000467       0x22 d:/ahl-gec-ide(4.26)º¬python/gcc/bin/../lib/gcc/arm-none-eabi/7.2.1/thumb/v7e-m/fpv4-sp/hard\libgcc.a(_arm_cmpdf2.o)
 .ARM.attributes
                0x00000489       0x22 d:/ahl-gec-ide(4.26)º¬python/gcc/bin/../lib/gcc/arm-none-eabi/7.2.1/thumb/v7e-m/fpv4-sp/hard\libgcc.a(_arm_fixunsdfsi.o)
 .ARM.attributes
                0x000004ab       0x22 d:/ahl-gec-ide(4.26)º¬python/gcc/bin/../lib/gcc/arm-none-eabi/7.2.1/thumb/v7e-m/fpv4-sp/hard\libgcc.a(_aeabi_uldivmod.o)
 .ARM.attributes
                0x000004cd       0x34 d:/ahl-gec-ide(4.26)º¬python/gcc/bin/../lib/gcc/arm-none-eabi/7.2.1/thumb/v7e-m/fpv4-sp/hard\libgcc.a(_fixunsdfdi.o)
 .ARM.attributes
                0x00000501       0x34 d:/ahl-gec-ide(4.26)º¬python/gcc/bin/../lib/gcc/arm-none-eabi/7.2.1/thumb/v7e-m/fpv4-sp/hard\libgcc.a(_udivmoddi4.o)
 .ARM.attributes
                0x00000535       0x22 d:/ahl-gec-ide(4.26)º¬python/gcc/bin/../lib/gcc/arm-none-eabi/7.2.1/thumb/v7e-m/fpv4-sp/hard\libgcc.a(_dvmd_tls.o)
 .ARM.attributes
                0x00000557       0x34 d:/ahl-gec-ide(4.26)º¬python/gcc/bin/../lib/gcc/arm-none-eabi/7.2.1/../../../../arm-none-eabi/lib/thumb/v7e-m/fpv4-sp/hard\libnosys.a(_exit.o)
 .ARM.attributes
                0x0000058b       0x34 d:/ahl-gec-ide(4.26)º¬python/gcc/bin/../lib/gcc/arm-none-eabi/7.2.1/thumb/v7e-m/fpv4-sp/hard/crtend.o
 .ARM.attributes
                0x000005bf       0x22 d:/ahl-gec-ide(4.26)º¬python/gcc/bin/../lib/gcc/arm-none-eabi/7.2.1/thumb/v7e-m/fpv4-sp/hard/crtn.o

.comment        0x00000000       0x7e
 .comment       0x00000000       0x7e ./obj/emuart.o
                                 0x7f (size before relaxing)
 .comment       0x0000007e       0x7f ./obj/system_msp432p401r.o
 .comment       0x0000007e       0x7f ./obj/startup_msp432p401r_gcc.o
 .comment       0x0000007e       0x7f ./obj/main.o
 .comment       0x0000007e       0x7f ./obj/flash.o
 .comment       0x0000007e       0x7f ./obj/gpio.o
 .comment       0x0000007e       0x7f ./obj/gec.o
 .comment       0x0000007e       0x7f ./obj/uart.o
 .comment       0x0000007e       0x7f ./obj/isr.o
 .comment       0x0000007e       0x7f ./obj/printf.o

.debug_info     0x00000000     0x8b52
 .debug_info    0x00000000      0xc8f ./obj/emuart.o
 .debug_info    0x00000c8f      0xd6a ./obj/system_msp432p401r.o
 .debug_info    0x000019f9      0xa56 ./obj/startup_msp432p401r_gcc.o
 .debug_info    0x0000244f      0xa14 ./obj/main.o
 .debug_info    0x00002e63     0x1096 ./obj/flash.o
 .debug_info    0x00003ef9     0x1547 ./obj/gpio.o
 .debug_info    0x00005440      0xc2d ./obj/gec.o
 .debug_info    0x0000606d     0x11f6 ./obj/uart.o
 .debug_info    0x00007263      0xa2d ./obj/isr.o
 .debug_info    0x00007c90      0xec2 ./obj/printf.o

.debug_abbrev   0x00000000     0x1746
 .debug_abbrev  0x00000000      0x29d ./obj/emuart.o
 .debug_abbrev  0x0000029d      0x115 ./obj/system_msp432p401r.o
 .debug_abbrev  0x000003b2      0x201 ./obj/startup_msp432p401r_gcc.o
 .debug_abbrev  0x000005b3      0x1f6 ./obj/main.o
 .debug_abbrev  0x000007a9      0x279 ./obj/flash.o
 .debug_abbrev  0x00000a22      0x308 ./obj/gpio.o
 .debug_abbrev  0x00000d2a      0x24b ./obj/gec.o
 .debug_abbrev  0x00000f75      0x2fe ./obj/uart.o
 .debug_abbrev  0x00001273      0x21f ./obj/isr.o
 .debug_abbrev  0x00001492      0x2b4 ./obj/printf.o

.debug_aranges  0x00000000      0x140
 .debug_aranges
                0x00000000       0x20 ./obj/emuart.o
 .debug_aranges
                0x00000020       0x20 ./obj/system_msp432p401r.o
 .debug_aranges
                0x00000040       0x20 ./obj/startup_msp432p401r_gcc.o
 .debug_aranges
                0x00000060       0x20 ./obj/main.o
 .debug_aranges
                0x00000080       0x20 ./obj/flash.o
 .debug_aranges
                0x000000a0       0x20 ./obj/gpio.o
 .debug_aranges
                0x000000c0       0x20 ./obj/gec.o
 .debug_aranges
                0x000000e0       0x20 ./obj/uart.o
 .debug_aranges
                0x00000100       0x20 ./obj/isr.o
 .debug_aranges
                0x00000120       0x20 ./obj/printf.o

.debug_line     0x00000000     0x2588
 .debug_line    0x00000000      0x35f ./obj/emuart.o
 .debug_line    0x0000035f      0x2ac ./obj/system_msp432p401r.o
 .debug_line    0x0000060b      0x3c6 ./obj/startup_msp432p401r_gcc.o
 .debug_line    0x000009d1      0x3dc ./obj/main.o
 .debug_line    0x00000dad      0x3ef ./obj/flash.o
 .debug_line    0x0000119c      0x3d4 ./obj/gpio.o
 .debug_line    0x00001570      0x419 ./obj/gec.o
 .debug_line    0x00001989      0x351 ./obj/uart.o
 .debug_line    0x00001cda      0x3e4 ./obj/isr.o
 .debug_line    0x000020be      0x4ca ./obj/printf.o

.debug_str      0x00000000     0x18e0
 .debug_str     0x00000000      0x683 ./obj/emuart.o
                                0x71d (size before relaxing)
 .debug_str     0x00000683      0x8c9 ./obj/system_msp432p401r.o
                                0xb02 (size before relaxing)
 .debug_str     0x00000f4c       0xea ./obj/startup_msp432p401r_gcc.o
                                0x6f6 (size before relaxing)
 .debug_str     0x00001036       0x4d ./obj/main.o
                                0x69a (size before relaxing)
 .debug_str     0x00001083       0xe0 ./obj/flash.o
                                0xa27 (size before relaxing)
 .debug_str     0x00001163      0x499 ./obj/gpio.o
                                0xb1f (size before relaxing)
 .debug_str     0x000015fc       0x42 ./obj/gec.o
                                0x704 (size before relaxing)
 .debug_str     0x0000163e       0xf7 ./obj/uart.o
                                0xaaa (size before relaxing)
 .debug_str     0x00001735       0x52 ./obj/isr.o
                                0x6bf (size before relaxing)
 .debug_str     0x00001787      0x159 ./obj/printf.o
                                0x776 (size before relaxing)

.debug_frame    0x00000000      0xd88
 .debug_frame   0x00000000      0x150 ./obj/emuart.o
 .debug_frame   0x00000150       0x60 ./obj/system_msp432p401r.o
 .debug_frame   0x000001b0       0x54 ./obj/startup_msp432p401r_gcc.o
 .debug_frame   0x00000204       0x30 ./obj/main.o
 .debug_frame   0x00000234      0x19c ./obj/flash.o
 .debug_frame   0x000003d0      0x1c8 ./obj/gpio.o
 .debug_frame   0x00000598       0x84 ./obj/gec.o
 .debug_frame   0x0000061c      0x21c ./obj/uart.o
 .debug_frame   0x00000838       0x60 ./obj/isr.o
 .debug_frame   0x00000898      0x17c ./obj/printf.o
 .debug_frame   0x00000a14       0x28 d:/ahl-gec-ide(4.26)º¬python/gcc/bin/../lib/gcc/arm-none-eabi/7.2.1/../../../../arm-none-eabi/lib/thumb/v7e-m/fpv4-sp/hard\libc_nano.a(lib_a-exit.o)
 .debug_frame   0x00000a3c       0x2c d:/ahl-gec-ide(4.26)º¬python/gcc/bin/../lib/gcc/arm-none-eabi/7.2.1/../../../../arm-none-eabi/lib/thumb/v7e-m/fpv4-sp/hard\libc_nano.a(lib_a-init.o)
 .debug_frame   0x00000a68       0x28 d:/ahl-gec-ide(4.26)º¬python/gcc/bin/../lib/gcc/arm-none-eabi/7.2.1/../../../../arm-none-eabi/lib/thumb/v7e-m/fpv4-sp/hard\libc_nano.a(lib_a-memcpy-stub.o)
 .debug_frame   0x00000a90       0x20 d:/ahl-gec-ide(4.26)º¬python/gcc/bin/../lib/gcc/arm-none-eabi/7.2.1/../../../../arm-none-eabi/lib/thumb/v7e-m/fpv4-sp/hard\libc_nano.a(lib_a-memset.o)
 .debug_frame   0x00000ab0       0x20 d:/ahl-gec-ide(4.26)º¬python/gcc/bin/../lib/gcc/arm-none-eabi/7.2.1/../../../../arm-none-eabi/lib/thumb/v7e-m/fpv4-sp/hard\libc_nano.a(lib_a-strcmp.o)
 .debug_frame   0x00000ad0       0x28 d:/ahl-gec-ide(4.26)º¬python/gcc/bin/../lib/gcc/arm-none-eabi/7.2.1/../../../../arm-none-eabi/lib/thumb/v7e-m/fpv4-sp/hard\libc_nano.a(lib_a-strncmp.o)
 .debug_frame   0x00000af8       0xac d:/ahl-gec-ide(4.26)º¬python/gcc/bin/../lib/gcc/arm-none-eabi/7.2.1/thumb/v7e-m/fpv4-sp/hard\libgcc.a(_arm_addsubdf3.o)
 .debug_frame   0x00000ba4       0x50 d:/ahl-gec-ide(4.26)º¬python/gcc/bin/../lib/gcc/arm-none-eabi/7.2.1/thumb/v7e-m/fpv4-sp/hard\libgcc.a(_arm_muldivdf3.o)
 .debug_frame   0x00000bf4       0xc4 d:/ahl-gec-ide(4.26)º¬python/gcc/bin/../lib/gcc/arm-none-eabi/7.2.1/thumb/v7e-m/fpv4-sp/hard\libgcc.a(_arm_cmpdf2.o)
 .debug_frame   0x00000cb8       0x24 d:/ahl-gec-ide(4.26)º¬python/gcc/bin/../lib/gcc/arm-none-eabi/7.2.1/thumb/v7e-m/fpv4-sp/hard\libgcc.a(_arm_fixunsdfsi.o)
 .debug_frame   0x00000cdc       0x2c d:/ahl-gec-ide(4.26)º¬python/gcc/bin/../lib/gcc/arm-none-eabi/7.2.1/thumb/v7e-m/fpv4-sp/hard\libgcc.a(_aeabi_uldivmod.o)
 .debug_frame   0x00000d08       0x2c d:/ahl-gec-ide(4.26)º¬python/gcc/bin/../lib/gcc/arm-none-eabi/7.2.1/thumb/v7e-m/fpv4-sp/hard\libgcc.a(_fixunsdfdi.o)
 .debug_frame   0x00000d34       0x34 d:/ahl-gec-ide(4.26)º¬python/gcc/bin/../lib/gcc/arm-none-eabi/7.2.1/thumb/v7e-m/fpv4-sp/hard\libgcc.a(_udivmoddi4.o)
 .debug_frame   0x00000d68       0x20 d:/ahl-gec-ide(4.26)º¬python/gcc/bin/../lib/gcc/arm-none-eabi/7.2.1/../../../../arm-none-eabi/lib/thumb/v7e-m/fpv4-sp/hard\libnosys.a(_exit.o)
